:020000040000FA
:100000004BEF0AF01200010034150000000F000051
:100010005400000046EC05F0FB0EDBCFF3FFDB06DF
:10002000F35000090AE094EC05F0FA0EFFEC05F03D
:10003000F3E1151CF1E1010E01D0000E75EF05F0A2
:1000400046EC05F03B0EE12402E3E168E652E16E86
:10005000010EDB6A020EDB6AF90EDBCFF6FFFA0E49
:10006000DBCFF7FFFB0EDBCFF8FF0800F550DF6EAC
:10007000DF5002E199EF04F0250EDF5C02E08CEF27
:1000800004F0030EDB6A040EDB6A050EDB6A060E63
:10009000DB6A070EDB6AAEEC04F02D0EDF5C0CE0D1
:1000A0002B0EDF5C09E0200EDF5C06E0230EDF5C38
:1000B00003E0300EDF5C1AE1DF50300A14E0130A6F
:1000C0000FE0030A0AE00B0A05E0060AE4E1030E6A
:1000D000DB80E1D7030EDB82DED7030EDB84DBD7C8
:1000E000030EDB86D8D7030EDB88D5D72A0EDF5C5C
:1000F0001BE1AAEC04F0F8EC04F010E0030EDB8046
:1001000008680968130EDBCF0DF0140EDBCF0EF07C
:10011000C1EC09F0040E06C0DBFF03D0130EE1ECC6
:1001200004F0AEEC04F00BD0090EDB6A4FEC05F0E6
:1001300003E0C3EC05F0FAD7090EE1EC04F0030E7E
:10014000DBB0DB982E0EDF5C1BE1AEEC04F02A0E78
:10015000DF5C0BE1AAEC04F0F8EC04F003E1130E11
:1001600033EC05F0AEEC04F00BD0090EDB6A4FEC7B
:1001700005F003E0C3EC05F0FAD7090E33EC05F007
:10018000680EDF5C07E1AEEC04F0680EDF5C1DE199
:10019000030E18D0740EDF5C17E07A0EDF5C14E0FB
:1001A000480EDF5C06E0540EDF5C03E05A0EDF5CB5
:1001B00002E1020E07D06C0EDF5C03E06A0EDF5C2A
:1001C00004E1010E86EC05F0C9DBDF506E0A01E1A7
:1001D0007FD31E0A01E192D1200A01E18FD13F0AAB
:1001E00001E149D11A0A01E146D10D0A01E143D1E9
:1001F000200A01E140D13A0A01E13DD1200A01E1A2
:100200003AD1260A01E135D10D0A01E132D11A0AAB
:1002100001E1D9D0200A4AE0300A1FE0460A0EE088
:10022000250A01E083D3D950F90FE96EFF0EDA20D9
:10023000EA6E010EEE5E000EEE5AEE5A94EC05F0F8
:10024000250EE66E95DB03E1151C01E169D390EC08
:1002500005F001E26BD3DB2A69D3080EDB6A040EDA
:10026000DB50010806E2040EDB0458EC05F0DB501D
:100270008BDB080EDB5009E0030EDB50010B05E1C0
:1002800072DB01E04DD3080EDB6A64DBEFCFDFFFEA
:1002900008EC06F003E1151C01E142D390EC05F0F7
:1002A00001E3DB2A60DB01E141D33AD3070EDB50E7
:1002B00002080FE1D4EC05F0030E9BEC05F00E0EE6
:1002C000EECFDBFF0F0EEECFDBFF100EEECFDBFF2E
:1002D00020D0F70EDBCF17F0F80EDBCF18F0020EB0
:1002E000175E000E185AF70E17C0DBFFF80E18C085
:1002F000DBFF17C0E9FF18C0EAFF8BEC05F0166AB8
:100300000E0E14C0DBFF0F0E15C0DBFF100E16C063
:10031000DBFF0E0EDBCFE6FF0F0EDBCFE6FF100E8E
:10032000DBCFE6FF9CEC09F0E552E552E552130EF7
:1003300007C0DBFF140E08C0DBFF060EDB5005E034
:10034000130ECFEC05F001E26ADBF3EC05F002E2FC
:10035000130E37DBB6EC05F006E0040ECFEC05F02B
:1003600002E2050E2EDB030EDBB005D0FCDA01E065
:10037000D7D2080EDB6A090EDB6A0E0EDBCFF6FF62
:100380000F0EDBCFF7FF100EDBCFF8FF0800F550A4
:10039000DF6EDF5014E0F9EC05F011E208EC06F036
:1003A00003E1151C01E1BCD2BBDB01E3DB2A090E32
:1003B000DB2AD9500E0FE96E000ECBDBE7D7D3DA7C
:1003C00001E1B4D2ADD2C6DA110EEECFDBFF120ED0
:1003D000EDCFDBFF110EDBCFE6FF120EDBCFE6FF2A
:1003E0008EEC09F0E552E552130EF3CFDBFF140E4D
:1003F000F4CFDBFF060EDB5004E0130ED0DB01E28E
:100400000EDBF3EC05F002E2130EDBDAAFDB05E006
:10041000040EC5DB02E2050ED4DA030EDBB005D014
:10042000A2DA01E07DD2080EDB6A090EDB6A110E4A
:10043000DBCFE9FF120EDBCFEAFFEFCFDFFFDF50AC
:1004400014E0D7DB12E2E4DB03E1151C01E168D222
:1004500067DB01E3DB2A090EDB2A110EDB2ADBCF87
:10046000E9FF120EE8E3DB2AE6D77DDA01E15ED28E
:1004700057D2030EDB8E070EDB0410E195DB040E72
:100480005ADB0A0EEECFDBFF0B0EEECFDBFF0C0EBE
:10049000EECFDBFF0D0EEECFDBFF6CD0070EDB5097
:1004A00003082CE1030EDBAE0DD0B2DA020E76DAD1
:1004B000EFCF14F0156A166A176A14AE39D01568B2
:1004C000166835D0F70EDBCF15F0F80EDBCF16F03F
:1004D000020E155E000E165AF70E15C0DBFFF80E61
:1004E00016C0DBFF15C0E9FF16C0EAFFEFCF14F01E
:1004F0000A0E14C0DBFF0B0EDB6A38D0070EDB5090
:10050000020809E1030EDBAE04D059DB16AE10D0B1
:100510000ED055DB0DD0030EDBAE12D079DA020E11
:100520003DDAF9DA166A176A15AE02D0166817684E
:10053000E2DA0C0E16C0DBFF0D0E17C0DBFF1AD07F
:10054000F70EDBCF16F0F80EDBCF17F0020E165EBB
:10055000000E175AF70E16C0DBFFF80E17C0DBFFB0
:1005600016C0E9FF17C0EAFFD6DAC5DA0C0EDB6A5F
:100570000D0EDB6A060EDB5005E1010EF36E050E73
:10058000F3CFDBFF150EDB6A160EDB6AD950370F8F
:10059000146E000EDA20156E390E14C0DBFF3A0E11
:1005A00015C0DBFF380EDB6A080EDB6A0A0EAEDA16
:1005B000DF50780A12E0200A10E0280A0CE0200A36
:1005C0000AE03F0A06E00D0A02E0200A08E1020EF6
:1005D00005D0080E03D0080EDF26100E97DA030EA2
:1005E000DBBE02D0DB92DB94DB50800B24E08ADAA6
:1005F000D890030EEB50000A08E6000EEE5C000EE9
:10060000EE58000EEE58000EEE5815E213DA0B68A5
:100610000C680D680E6856EC09F00A0E02C0DBFF8C
:100620000B0E03C0DBFF0C0E04C0DBFF0D0E05C07C
:10063000DBFF2D0E08D0030EDBA202D02B0E03D061
:10064000DBA408D0200EF36E170EF3CFDBFF150EE0
:10065000DB2A02D0170EDB6A050EDB5003E1B7D9A7
:1006600001E189D0100E146E150E156E000E166E77
:10067000070EDBCF17F0186A196A1A6A17C00BF059
:1006800018C00CF019C00DF01AC00EF0D3D9EEEC62
:1006900009F014500224F36E15500320F46E165026
:1006A0000420F86EF4CFF7FFF3CFF6FF0800090E31
:1006B000F5CFDBFF580EDF5C0FE1610EF36E090E24
:1006C0007BD90AE3200E146E090EDBCFE7FF14502E
:1006D000E75E090EE7CFDBFF070EDBCF14F0156AEC
:1006E000166A176A0FDA14C00BF015C00CF016C0AA
:1006F0000DF017C00EF0EECF06F0EECF07F0EECF04
:1007000008F0EFCF09F0EEEC09F009C0EDFF08C0EA
:10071000EDFF07C0EDFF06C0EFFF390EDBCFE9FFAD
:10072000DB063A0EDBCFEAFF01E2DB06090EDBCF88
:10073000EFFF150EDB2A4BD995E1030EDBA61DD08A
:100740006F0EDF5C06E1C1D918E3150EDB285BDA1A
:1007500014D0780EDF5C09E0580EDF5C06E0620E14
:10076000DF5C03E0420EDF5C08E1020EF36E160E62
:10077000F3CFDBFF02D0150EDB6A030EDB50100B4C
:100780000EE0040EDBCF14F0050EDB50D8801454BD
:1007900006E2060EDB5003E1040EDB5034DA95D995
:1007A0000AE2050EDBCFE7FF150EDB50E75E050E14
:1007B000E7CFDBFF02D0050EDB6A040EDBCF14F0BF
:1007C000160E45D9D880145414E2160EDBCFE6FF7E
:1007D000150EDBCFE6FF040EDBCFE6FF050EDB5088
:1007E000E552E75CE552D880E754E552D880E754FB
:1007F0005FD9030EDB50010B0BE1080EDB5008E064
:10080000B2D801E08DD0080EDB50BED8080EDB6AEE
:10081000170EDB5007E088D9170EF1D903E1151C3C
:1008200001E17ED0160EDB5016E07ED9300EE66E6A
:100830009FD802E1151C74E077D9DFCFE6FF14ECF6
:1008400009F0E552E552E552F4CF15F00001F31C32
:1008500002E1151C65E0050EDBCF14F0160EDB502F
:10086000D880145409E2050EDBCFE7FF160EDB50EB
:10087000E75E050EE7CFDBFF300EE66E050ECBD947
:100880004FE1390EDB2ADBCFE9FF3A0E01E3DB2A29
:10089000DBCFEAFF090EEFCFDBFFDB500EE044D9E0
:1008A000090EADD902E1151C3BE0390EDB2ADBCF86
:1008B000E9FF3A0EEDE3DB2AEBD755D831E1160E0E
:1008C000DBCFE6FF080EC3D8E552E7245DD82ED073
:1008D000070EDB50030A1CE0010A14E0030A07E0DC
:1008E0007BD9DBCFEEFF020EDBCFEDFF1FD0F5D8BB
:1008F000196A17AE02D0186819682CD8BCD819C06C
:10090000EEFF14D0EAD817BE186824D8B4D80ED099
:1009100063D9DBCFEFFF0AD07BD905E1151C03E1DA
:10092000F368F46810D0FCD801E3DB2A79D935EFFD
:1009300000F0010EDBCF14F0020EDBCF15F014C077
:10094000F3FF15C0F4FF3B0EE15C02E2E16AE55201
:10095000E16ECBD029D9020E9BEF05F061D90800DA
:10096000F550DF6E1200200EE66E080E0BEF06F05B
:1009700014EC09F0E552E552E552F3CF14F0F4CF50
:1009800015F00001F31C1200146E156AD950010F06
:100990004DD91450EE261550ED221200185E000EAF
:1009A000195AF70E18C0DBFFF80E19C0DBFF18C08C
:1009B000E9FF19C0EAFF1200DBCFF4FFF350F45C4B
:1009C0001200DB50E76E040EE7CFDBFF12000A0EC9
:1009D000DBCF14F00B0EDBCF15F00C0EDBCF16F0D7
:1009E0000D0EDBCF17F01450151016101710120053
:1009F000130EEECFDBFF140EEDCFDBFF130EDBCFBC
:100A000014F0140EDBCF15F00001800E1514120047
:100A1000F70EDBCF18F0F80EDBCF19F01200050E41
:100A2000DB50E66ED950130F01D9E552E750EE6E58
:100A3000ED6A12000A0EDBCF06F00B0EDBCF07F0DB
:100A40000C0EDBCF08F00D0EDBCF09F01200DBCF70
:100A5000E6FF150EDBCFE6FF050EDB50E552E7247F
:100A6000E552E7241200DB50CED8010EF36E060EDD
:100A7000F3CFDBFF1200EE50EFCFEAFFE96E16C0B6
:100A8000EEFF17C0EEFF18C0EEFF1200D9CFE6FF51
:100A9000DACFE6FFE1CFD9FFE2CFDAFF1200DFCFF6
:100AA000E6FFE66A29EC0AF0E552E552F35012003F
:100AB000E76E080EE7CFDBFF1200EECF14F0EECFAB
:100AC00015F0EFCF16F0176A1200050EDBCF14F009
:100AD000150EDB50D88014541200010EDBCF16F037
:100AE000020EDBCF17F0186A1200E552E5CFDAFFED
:100AF000E7CFD9FF12000A0E14C0DBFF0B0E15C0A2
:100B0000DBFF1200D9500A0F16EF06F0F36E070E46
:100B1000F3CFDBFF1200EECF14F0EFCF15F0120091
:100B2000010EDB2A020E1200FC0EDBCFE6FFFD0EEB
:100B3000DBCFE6FF1200145E000E155AF70E14C04C
:100B4000DBFFF80E15C0DBFF14C0E9FF15C0EAFF9C
:100B50001200DA20EA6EEF2AEECFF6FF000EEF2247
:100B6000EECFF7FFEF22EECFF8FF1200040EDBCF3F
:100B7000E6FF130EDB50E552E75C9ADFDB5004DF43
:100B8000060EDB501200090EDB500A0DF350DF2475
:100B9000D00FE76E090EE7CFDBFFAEEF04F0DB50BE
:100BA000F36E050EDCEF04F0F70EDBCF14F0F80E59
:100BB000DBCF15F01200DFCFE6FFB8EF04F028DF3F
:100BC000030EECDE5DEF05F00AEC00F0E552E552B5
:100BD000E552E55200091200BDDEEE50EFCFEAFF0C
:100BE000E96E010E1200130EDB50F36E040EDCEF03
:100BF00004F0040EDB50F36E090EDCEF04F0DBCFE3
:100C0000E6FFB8EF04F0E76E050EE7CFDBFF12005A
:100C10008BDFDBEF05F0DBCFE6FF86DFE4EF05F0EF
:100C2000D950F90FE96EFF0EA9EF05F0E96E000E3D
:100C3000DA20EA6E12000F0E9316811693949396A3
:100C400081948196F6D80F0E8116300E811227D826
:100C500015D90F0E8116300E811221D80FD90F0E23
:100C60008116300E81121BD809D90F0E8116818A88
:100C700016D8280EE66E17D8E552080EE66E13D881
:100C8000E552010EE66E0FD8E552060EE66E0BD861
:100C9000E5520F0EE66E07D8E55200D012008186AD
:100CA00012D981961200D9CFE6FFE1CFD9FF0FD933
:100CB000819481960F0E8116FE0EDB50F00B81128F
:100CC000EEDF0F0E8116FE0EDB38F00BF00B8112FB
:100CD000E6DF00D0E552E7CFD9FF1200D9CFE6FF1B
:100CE000E1CFD9FFF4D8818481960F0E8116FE0ED4
:100CF000DB50F00B81128186E6D881960F0E8116AB
:100D0000FE0EDB38F00BF00B81128186DCD8819669
:100D100000D0E552E7CFD9FF1200D9CFE6FFE1CFEF
:100D2000D9FFFD0EDBCFF6FFFE0EDBCFF7FF08008D
:100D3000F55011E0FD0EDBCFF6FFFE0EDBCFF7FF27
:100D40000800F550E66ECADFE552FD0EDB2AFE0E06
:100D500001E3DB2AE6D700D0E552E7CFD9FF120046
:100D6000D9CFE6FFE1CFD9FFFD0EDBCFE9FFFE0EC5
:100D7000DBCFEAFFEF5010E0FD0EDBCFE9FFFE0E08
:100D8000DBCFEAFFEF50E66EA9DFE552FD0EDB2A6E
:100D9000FE0E01E3DB2AE8D700D0E552E7CFD9FF0A
:100DA0001200D9CFE6FFE1CFD9FFE652FE0EDB04F9
:100DB00004E1FD0EDB50800FDF6EFE0EDB500208FB
:100DC00004E1FD0EDB50C00FDF6EDFCFE6FF6BDF0F
:100DD000E552E552E552E7CFD9FF1200D9CFE6FF41
:100DE000E1CFD9FFE652E66AFE0EDBCFE6FFD9DFA0
:100DF000E552E552DF6ADFCF14F0100EE76E1418EB
:100E0000E8AE02D0E73402D0E750145C06E2200ED0
:100E1000E66E64DFE552DF2AEED7E66AFE0EDBCF30
:100E2000E6FFBFDFE552E552E552E552E7CFD9FFD5
:100E30001200D9CFE6FFE1CFD9FF020EE126DE6A2C
:100E4000DD6ADECF14F0DDCF15F0D890155004E642
:100E5000100E145C270E155806E20000DF2A010E62
:100E600001E3DB2AEED700D0020EE15C02E2E16A88
:100E7000E552E16EE552E7CFD9FF1200D9CFE6FF88
:100E8000E1CFD9FF020EE126DE6ADD6ADECF14F083
:100E9000DDCF15F0D890155004E6C40E145C090E91
:100EA000155806E20000DF2A010E01E3DB2AEED727
:100EB00000D0020EE15C02E2E16AE552E16EE55229
:100EC000E7CFD9FF12000000000000001200D9CFC8
:100ED000E6FFE1CFD9FF020EE126DE6ADD6ADECF52
:100EE00014F0DDCF15F0D890155004E6E80E145C30
:100EF000030E155806E20000DF2A010E01E3DB2A8B
:100F0000EED700D0020EE15C02E2E16AE552E16E4A
:100F1000E552E7CFD9FF1200D9CFE6FFE1CFD9FFE5
:100F2000020EE126FD0EDBCF14F0FE0EDBCF15F036
:100F3000D89014361536D89014361536010E142470
:100F4000C26E0A0EE66E74EC0AF0E55296EC0AF0F8
:100F500091EC0AF0000901E0FBD77FEC0AF0F3CF37
:100F6000DEFFF4CFDDFFDECF14F0DDCF15F014C0CF
:100F7000F3FF15C0F4FF020EE15C03E200D0E16A6A
:100F8000E552E16EE552E7CFD9FF12008168936A1E
:100F90007F6AF19E7C687E6A7E807E82896A0F0EFF
:100FA000926E806A8268BF0E946E9480948294845C
:100FB00094869488948A949C948ED08ED09C786ADF
:100FC0001200C280C19AC198C08EC08AC088C096E3
:100FD000C084C092C0801200D9DFF3DF8998FA0E76
:100FE000E66E12EC0AF0E552898825DE010EE66E07
:100FF000F5DEE552DE0EE66E140EE66E8EDEE5528E
:10100000E552FA0EE66E12EC0AF0E552020EE66EBA
:10101000E5DEE552480EE66E61DEE552450EE66E0F
:101020005DDEE5524C0EE66E59DEE5524C0EE66E84
:1010300055DEE5524C0EE66E51DEE5524F0EE66E81
:101040004DDEE552FA0EE66E12EC0AF0E552020EA3
:10105000E66EC4DEE552D30EE66E140EE66E5DDE7D
:10106000E552E5528978000EE66EE66A55DFE552F4
:10107000E552F3CF96F0F4CF97F096C0E6FF97C015
:10108000E6FFCE0E146E140E156E166A14C0E6FF3F
:1010900015C0E6FF16C0E6FF52CFE6FF53CFE6FFCE
:1010A0006FEC08F0176E070EE15E1750F3CF64F097
:1010B000F4CF65F00B0EE66E020EE66E72DEE552C0
:1010C000E55252CFE6FF53CFE6FF4ADEE552E55246
:1010D000960EE66E12EC0AF0E552C4D71200D9CF94
:1010E000E6FFDACFE6FFE1CFD9FFE2CFDAFFE65243
:1010F000E652E652E652D950F90F146EFF0EDA208E
:10110000156E020E14C0DBFF030E15C0DBFF020ECE
:10111000DBCFE6FF030EDBCFE6FFF90EDBCFE6FF0A
:10112000FA0EDBCFE6FFFB0EDBCFE6FFD950FC0F5C
:10113000E66EFF0EDA20E66E20EC00F0146E070E6D
:10114000E15C02E2E16AE552E16E1450F3CFDEFFAA
:10115000F4CFDDFFFC0EDBCFE9FFFD0EDBCFEAFFB6
:10116000EF6ADECF14F0DDCF15F014C0F3FF15C029
:10117000F4FF040EE15C02E2E16AE552E16EE55241
:10118000E5CFDAFFE7CFD9FF1200060EF66E000EAC
:10119000F76E000EF86E0F010900F550596F090047
:1011A000F5505A6F03E1596701D03DD00900F55061
:1011B000546F0900F550556F0900F550566F09003E
:1011C0000900F550E96E0900F550EA6E09000900C2
:1011D0000900F550576F0900F550586F09000900D4
:1011E000F6CF5BFFF7CF5CFFF8CF5DFF54CFF6FF84
:1011F00055CFF7FF56CFF8FF0F01575302E1585371
:1012000007E00900F550EE6E5707F8E25807F9D7E6
:101210005BCFF6FF5CCFF7FF5DCFF8FF0F015907FB
:10122000000E5A5BBFD71200D9CFE6FFDACFE6FF38
:10123000E1CFD9FFE2CFDAFFFB0EDBCF14F0FC0EDB
:10124000DBCF15F00001800E15141AE1FB0EDBCF89
:10125000E9FFFC0EDBCFEAFFEECFF3FFEDCFF4FFAB
:10126000EE2A000EEF22F3CFE9FFF4CFEAFFFD0EE6
:10127000DBCFEFFFEF50156AF36E15C0F4FF10D00F
:10128000FB0EDB50FE0806E1FD0EDBCFE6FF59EC5E
:101290000AF005D0FD0EDBCFE6FF98EC0AF0E55230
:1012A000E552E5CFDAFFE7CFD9FF120006500B0277
:1012B000F3CF02F0F4CF03F00C02F3500326000E3C
:1012C000F420046E06500D02F3500426000EF420A4
:1012D000056E06500E02F350052607500B02F35020
:1012E0000326F4500422000E052207500C02F3508E
:1012F0000426F450052207500D02F350052608502D
:101300000B02F3500426F450052208500C02F3504F
:10131000052609500B02F35005261200FE0EE3CFFE
:10132000E9FFFF0EE3CFEAFFF36AF46AEE5203E04F
:10133000F34AF42AFBD71200FF0EE3CFF8FFE55281
:10134000FF0EE3CFF7FFE552FF0EE3CFF6FFE552C6
:10135000E66AE66AE66A0900F55209E0FD0EE32A4C
:1013600005E1FE0EE32A02E1FF0EE32AF4D7FD0EAB
:10137000E3CF07F0FE0EE3CF08F0FF0EE3CF09F056
:10138000120009C013F008C012F008500D02F4CF8B
:1013900007F0F3CF06F009500E02F4CF09F0F3CFB7
:1013A00008F00D02F3500726F4500822E86A0922DB
:1013B00012500E02F3500726F4500822E86A092260
:1013C0000EAEE7EF09F01250085E1350095A13AE43
:1013D000000C0D50085E0E50095A000C056A046A94
:1013E000036A026A200EE76ED89006360736083682
:1013F000093602360336043605360B50025C0C50B3
:1014000003580D5004580E50055809E30B50025E66
:101410000C50035A0D50045A0E50055A062AE72E56
:10142000E4D71200FF0EE3501C6EEF0E01D0F30E56
:10143000E76EE72E19EF0AF00C0E1B6EE76AE72E37
:101440001FEF0AF01B2E1EEF0AF01C2E17EF0AF0FA
:101450001200F36AF46AFF0EE124E96EFF0EE22047
:10146000EA6EED6607D02F0EEF6404D03A0EEF60FF
:1014700001D0F32A1200600EF36E00EE00F00F0EA2
:1014800001D81200EA6002D0EE6AFCD7F350E9609E
:101490001200EE6AFCD71EEE00F02EEE00F0F86AA5
:1014A000019CC5EC08F099EC0AF0ECEC07F0FBD7D6
:1014B0001200FF0EE350ACBA04D0AF6AAB8EAC8A18
:1014C000949CACA2FED7AD6EF36EF46A1200253088
:1014D0003464004D657375726520434830002020E8
:1014E00053414C5554202000FF0EE350E84E1200AB
:1014F000000000D000D000D0E82EFAD71200C4506F
:10150000176E166AC3501610F36E17C0F4FF120060
:101510003031323334353637383961626364656669
:1015200000FFC250020B01E0010E1200C282120045
:101530001200120031323334353637383930313217
:1015400033343500000F50524F4A45542043313850
:10155000203A31384632364B32785F4C4344327849
:1015600031362E6D63700D00000000000000000099
:10157000000000000000000000000000000000006B
:10158000000000000000120FFFFFFFFFFFFFFFFF42
:10159000FFFFFFFFFFFFFFFFFFFFFFFFFFFFFFFF5B
:1015A000FFFFFFFFFFFFFFFFFFFFFFFFFFFFFFFF4B
:1015B000FFFFFFFFFFFFFFFFFFFFFFFFFFFFFFFF3B
:1015C000FFFFFFFFFFFFFFFFFFFFFFFFFFFFFFFF2B
:0200000400F00A
:020000040030CA
:0E0000000008191E008980000FC00FE00F409D
:020000040020DA
:08000000FFFFFFFFFFFFFFFF00
:00000001FF
